:100000007B29B800E7200A30FE20380880048413DA
:100010008006A001A101841738088006640010281A
:1000200011281228132880068413000503191E289E
:100030002408A0070318A10F0B28A1032108762983
:100040006400362003182028A920A8010830A30046
:10005000AA2036200318A80AAB1EA801A20CA30BE5
:100060002828AB1AA213AA20220808003A08840004
:10007000380884178004841300052B1B3806FF3EC4
:100080000800A401A501B7127121D33E0319B716C8
:100090002D3EC63E031844280A3E031C4428A200F5
:1000A0000310240DA000250DA100200DA10DA40713
:1000B0000318A10A2108A507A40DA50D2208A4076D
:1000C0000318A50AA90303196C287121C63E031859
:1000D0006C280A3E03184F28B71E7328A409A509E7
:1000E000A40A0319A50A240876290408A6003A08D8
:1000F00084008030B7050830A70003100318B70A42
:100100008F20A60CA70B7E280000AB1A370C8F207F
:10011000792103148F202F08A3002E08FF288413B1
:10012000AB1F9E28000838042B1F38068000841758
:1001300000083804031C38068000AA280008380488
:10014000031C38062B1B38068000841738098005ED
:10015000AA2837172B081F39003EA1002A080E3E97
:100160000318A10A371F0C293713A00002301E21E3
:100170000C29B71329080319B7170530A800273031
:10018000A3001030CF200330A300E830CF20A3011C
:100190006430CF20A3010A30CF202408D628A20043
:1001A0002508A1002408A0003F212008A000A803E2
:1001B0000319B71329080319E028280203180800B7
:1001C0002008031DB713B71B0800303E71298004B7
:1001D000E928FF3A84178005762983169B001C14B2
:1001E0001A08762983169A001C1555309D00AA30EE
:1001F0009D009C149C18FA281C117629A301A200CA
:10020000FF30A207031CA307031C76290330A100BB
:10021000E6300C210029A101FC3EA000A109031C2D
:100220001729FF300000A00703181229A007640057
:10023000A10F112908000310A10CA00CFF3E031808
:100240001B2920087629A101A301A2000230282938
:10025000A80023082102031D2F29220820020430B0
:1002600003180130031902302805031DFF307629D9
:100270000038031DFF300405031DFF307629A5015A
:10028000A4011030A600210DA40DA50D2208A40282
:100290002308031C230FA502031855292208A407CD
:1002A00023080318230FA5070310A00DA10DA60B0B
:1002B0004329200876291030A800A101A001A70C2D
:1002C000A60C031C69292208A00723080318230F82
:1002D000A107A10CA00CA50CA40CA80B5F29240855
:1002E0007629840031088A003008820083130313C2
:1002F00083126400080007309F00831686170617D4
:100300008616061686150615861406140515051597
:1003100005168514051064008312051A9029402DD6
:100320008316851483127D265908A00031302321BD
:10033000B2000030861B0130A00001302321B40040
:100340003208840034083821B400B5006400340851
:1003500035040319072A4908A00031302321B200CF
:100360005108A00031302321B40032088400340841
:100370003821B400B5006400340835040319C229DB
:10038000BA24072A4908A00031302321B2005208BC
:10039000A00031302321B400320884003408382111
:1003A000B400B5006400340835040319D929D324F6
:1003B000072A4A08A00031302321B2005108A000CA
:1003C00031302321B4003208840034083821B400CD
:1003D000B5006400340835040319F029E924072A1C
:1003E0004A08A00031302321B2005208A000313069
:1003F0002321B4003208840034083821B400B50049
:100400006400340835040319072AFF24072A5A0810
:10041000A00031302321B2000030061B0130A000C3
:1004200001302321B4003208840034083821B4009C
:10043000B50064003408350403197A2A4908A0007D
:1004400031302321B2005108A00031302321B40003
:100450003208840034083821B400B5006400340840
:1004600035040319352ABA247A2A4908A000313004
:100470002321B2005208A00031302321B4003208F9
:10048000840034083821B400B50064003408350411
:1004900003194C2AD3247A2A4A08A0003130232198
:1004A000B2005108A00031302321B400320884008A
:1004B00034083821B400B500640034083504031949
:1004C000632AE9247A2A4A08A00031302321B200A5
:1004D0005208A00031302321B400320884003408CF
:1004E0003821B400B50064003408350403197A2AB1
:1004F000FF247A2A5B08A00031302321B2000030AB
:10050000861A0130A00001302321B4003208840093
:1005100034083821B400B5006400340835040319E8
:10052000ED2A4908A00031302321B2005108A00073
:1005300031302321B4003208840034083821B4005B
:10054000B5006400340835040319A82ABA24ED2A3A
:100550004908A00031302321B2005208A0003130F8
:100560002321B4003208840034083821B400B500D7
:100570006400340835040319BF2AD324ED2A4A083D
:10058000A00031302321B2005108A00031302321D6
:10059000B4003208840034083821B400B500640087
:1005A000340835040319D62AE924ED2A4A08A000A4
:1005B00031302321B2005208A00031302321B40091
:1005C0003208840034083821B400B50064003408CF
:1005D00035040319ED2AFF24ED2A5C08A000313010
:1005E0002321B2000030061A0130A000013023217F
:1005F000B4003208840034083821B400B500640027
:10060000340835040319602B4908A0003130232138
:10061000B2005108A00031302321B4003208840018
:1006200034083821B400B5006400340835040319D7
:100630001B2BBA24602B4908A00031302321B200C3
:100640005208A00031302321B4003208840034085D
:100650003821B400B5006400340835040319322B86
:10066000D324602B4A08A00031302321B200510866
:10067000A00031302321B40032088400340838212E
:10068000B400B5006400340835040319492BE9248B
:10069000602B4A08A00031302321B2005208A0008C
:1006A00031302321B4003208840034083821B400EA
:1006B000B5006400340835040319602BFF24602B57
:1006C0005D08A00031302321B200003086190130CE
:1006D000A00001302321B4003208840034083821FE
:1006E000B400B5006400340835040319D32B49085D
:1006F000A00031302321B2005108A0003130232165
:10070000B4003208840034083821B400B500640015
:100710003408350403198E2BBA24D32B4908A000C2
:1007200031302321B2005208A00031302321B4001F
:100730003208840034083821B400B500640034085D
:1007400035040319A52BD324D32B4A08A00031303C
:100750002321B2005108A00031302321B400320817
:10076000840034083821B400B5006400340835042E
:100770000319BC2BE924D32B4A08A00031302321D4
:10078000B2005208A00031302321B40032088400A6
:1007900034083821B400B500640034083504031966
:1007A000D32BFF24D32B5E08A00031302321B200CD
:1007B000003006190130A00001302321B4003208B6
:1007C000840034083821B400B500640034083504CE
:1007D0000319462C4908A00031302321B2005108EA
:1007E000A00031302321B4003208840034083821BD
:1007F000B400B5006400340835040319012CBA2490
:10080000462C4908A00031302321B2005208A00034
:1008100031302321B4003208840034083821B40078
:10082000B5006400340835040319182CD324462C71
:100830004A08A00031302321B2005108A000313015
:100840002321B4003208840034083821B400B500F4
:1008500064003408350403192F2CE924462C4A0877
:10086000A00031302321B2005208A00031302321F2
:10087000B4003208840034083821B400B5006400A4
:10088000340835040319462CFF24462C5F08A000C9
:1008900031302321B200003086180130A000013031
:1008A0002321B4003208840034083821B400B50094
:1008B0006400340835040319B92C4908A00031300C
:1008C0002321B2005108A00031302321B4003208A6
:1008D000840034083821B400B500640034083504BD
:1008E0000319742CBA24B92C4908A00031302321F3
:1008F000B2005208A00031302321B4003208840035
:1009000034083821B400B5006400340835040319F4
:100910008B2CD324B92C4A08A00031302321B200FB
:100920005108A00031302321B4003208840034087B
:100930003821B400B5006400340835040319A22C32
:10094000E924B92C4A08A00031302321B200520812
:10095000A00031302321B40032088400340838214B
:10096000B400B5006400340835040319B92CFF2421
:10097000B92C94293F08A3003E08FF2005148316D4
:100980000510831285108316851083124508A30075
:100990004408FF2005108316051083128514831662
:1009A0008510831208003F08A3003E08FF200514AD
:1009B000831605108312851083168510831229254E
:1009C0000510831605108312851483168510831273
:1009D000080012250514831605108312851083164E
:1009E000851083124508A3004408FF2005108316D4
:1009F00005108312851483168510831208001225B2
:100A00000514831605108312851083168510831232
:100A10002925051083160510831285148316851069
:100A2000831208004E08A400053084000430012021
:100A3000D7005708A600A7014008A2004108A3005C
:100A40005B21B2002508B3003308A3003208FF2061
:100A500008004F08A4000530840008300120D700AA
:100A60005708A600A7014608A2004708A3005B217B
:100A7000B2002508B3003308A3003208FF200800A5
:100A80000530BA001030B8005430AA00AB01202065
:100A9000243C031D472D2020D7002020D8002020F3
:100AA000D9002020DA002020DB002020DC002020DC
:100AB000DD002020DE002020DF002020E0000230CA
:100AC000A9002030B000B1014120D6002020CA008A
:100AD0000430A9002030B000B1014120C000250839
:100AE000C1002020C9000430A9002030B000B101AD
:100AF0004120BE002508BF002020CB002020CC00D4
:100B00002020CD002020C8000430A9002030B000F3
:100B1000B1014120BC002508BD002020D2000430D6
:100B2000A9002030B000B1014120C6002508C7004F
:100B30002020D1000430A9002030B000B1014120B4
:100B4000C4002508C5002020D3002020D400202088
:100B5000D5002020D0000430A9002030B000B10121
:100B60004120C2002508C30064005708343C031D1F
:100B7000E42D64005808573C031DBF2DE72E640088
:100B80005808523C031DC52DFF2D64005808453CF4
:100B9000031DCB2D942964005808503C031DD72D0C
:100BA000831621309B0083125908F220E52D640042
:100BB0005808513C031DE32D831622309B008312FD
:100BC0005908F220F22DE42D402D5908A4000530DB
:100BD000840004300120D700AE270130A300F43098
:100BE000FF20E52D5908A4000530840008300120BD
:100BF000D700AE270130A300F430FF20F22D7D2670
:100C00000530BA000230B8005430AA00AB01AE0182
:100C1000AF012430762057087620580876205908EE
:100C200076205A0876205B0876205C0876205D08DE
:100C300076205E0876205F087620600876200230F5
:100C4000A9005608A400A5017530B000B101B92073
:100C50004A0876200430A9004008A4004108A500F5
:100C60007530B000B101B920490876200430A900E0
:100C70003E08A4003F08A5007530B000B101B920BE
:100C80004B0876204C0876204D08762048087620C0
:100C90000430A9003C08A4003D08A5007530B00050
:100CA000B101B920520876200430A9004608A400FA
:100CB0004708A5007530B000B101B9205108762071
:100CC0000430A9004408A4004508A5007530B00010
:100CD000B101B920530876205408762055087620B3
:100CE000500876200430A9004208A4004308A5005B
:100CF0007530B000B101B920402D0030ED20D90091
:100D00000130ED20DA000230ED20DB000330ED2071
:100D1000DC000430ED20DD000530ED20DE00063083
:100D2000ED20DF000730ED20E0000830ED20D60098
:100D30000930ED20CA000A30ED20C0000B30ED2054
:100D4000C1000C30ED20C9000D30ED20BE000E308A
:100D5000ED20BF000F30ED20CB001030ED20CC0097
:100D60001130ED20CD001230ED20C8001330ED2001
:100D7000BC001430ED20BD001530ED20D20016303F
:100D8000ED20C6001730ED20C7001830ED20D1004F
:100D90001930ED20C4001A30ED20C5001B30ED20C5
:100DA000D3001C30ED20D4001D30ED20D5001E30C6
:100DB000ED20D0001F30ED20C2002030ED20C30018
:100DC0002130ED20CE002230ED20CF000800831628
:100DD0009B0183125908F220831601309B00831275
:100DE0005A08F220831602309B0083125B08F2201F
:100DF000831603309B0083125C08F22083160430B4
:100E00009B0083125D08F220831605309B0083123D
:100E10005E08F220831606309B0083125F08F220E2
:100E2000831607309B0083126008F2208316083077
:100E30009B0083125608F220831609309B00831210
:100E40004A08F22083160A309B0083124008F220E1
:100E500083160B309B0083124108F22083160C305E
:100E60009B0083124908F22083160D309B008312E9
:100E70003E08F22083160E309B0083123F08F220BA
:100E800083160F309B0083124B08F220831610301C
:100E90009B0083124C08F220831611309B008312B2
:100EA0004D08F220831612309B0083124808F2206E
:100EB000831613309B0083123C08F22083161430F3
:100EC0009B0083123D08F220831615309B0083128D
:100ED0005208F220831616309B0083124608F22037
:100EE000831617309B0083124708F22083161830B0
:100EF0009B0083125108F220831619309B00831245
:100F00004408F22083161A309B0083124508F22011
:100F100083161B309B0083125308F22083161C306B
:100F20009B0083125408F22083161D309B0083120D
:100F30005508F22083161E309B0083125008F220C1
:100F400083161F309B0083124208F2208316203044
:100F50009B0083124308F220AE27402D0530BA00D3
:100F60000230B8005430AA00AB01AE01AF0124300A
:080F70007620570876200800E6
:02400E002A3F47
:00000001FF
